S00600004844521B
S123B600CE000018CEB6D5C62918A600A7000818085AC10026F3CE010018CEB6FEC62918C7
S123B620A600A7000818085AC10026F3861ABDFFB88600B71009B6100884044444BDB6ADF5
S123B640971DB610088408444444BDB6AD9725B61008841044444444BDB6ADB7010DB61013
S123B6600884204444444444BDB6ADB701158614BDB6C9CE0000BDFFCABDB69BBDFFC4BD64
S123B680FFC48614BDB6C9CE0100BDFFCABDB69B860BBDFFB8BDFFB87EB63618CE0040861B
S123B6A008BDFFB81809188C000026F3394848484844444444840F8B3081392F028B0739BF
S123B6C0BDFFC45AC10026F839168620BDFFB85AC10026F83972656164696E672050443014
S123B6E03A204E43205044313A204E43205044323A202020205044333A202020200472658F
S123B7006164696E67205044343A202020205044353A202020205044363A204E4320504494
S10AB720373A204E432004D8
S9030000FC
